:1000000009C018951895189518951895189518956C
:10001000189518958FE98DBFC0EAE8EB4E2EDD27C5
:100020005D2EEEE3F0E0A0E6B0E088278D933197F7
:10003000E9F76624B99AB89ABC98BD98BA9A379AE3
:1000400080E08093640083E087B98ED0A0E68D9332
:100050009C93A0E60D911C91043652E0150710F018
:1000600009F001C021C000916400013009F002C014
:10007000C09A0EC0023009F002C0C19A09C0033014
:1000800009F002C0C09804C0043009F001C0C19852
:10009000C29800E014E0A0E64D915C91041B150BA2
:1000A000A2E60D931C9326C0A0E60D911C910C397D
:1000B00051E0150708F01DC000916400013009F0FF
:1000C00002C0C19A0EC0023009F002C0C09A09C035
:1000D000033009F002C0C19804C0043009F001C027
:1000E000C098C298A0E68D919C91A2E68D939C93B6
:1000F00001C0C29AA2E60D911C91083050E015078C
:1001000008F005C088E090E0A2E68D939C93A2E6FB
:100110008D919C911AD0A4E68C918F5F8C93009165
:100120006400043010F009F001C003C081E0809346
:10013000640089CFF894FFCF3197F1F70895689460
:1001400062F80895E89462F80895EF93FF93EE271C
:10015000E82BE92B31F0EDECFAE03197F1F701975C
:10016000D1F7FF91EF910895369A3699FECF369ADE
:0A0170003699FECF84B195B10895D1
:00000001FF
